S1048000007B
S123C000C73FC721C748C77CC727C72FC737C78AC7A2C79AC7AAC7FCC7F2C7E6C7EBC805C6
S123C020C81DC86BC82DC83DC84DC8F3C913C91FC933C745CA16C949C95EC953CA72CA7E95
S123C040CA89C97BC967C985C98FC99FC9E0CA0CCA1BCA37CA46CA55C9ECC9FCC9D1C9B7DF
S123C060CA9ECAA2CAA8CAB9CACCCABFCB02CAD4CB12CB75CB8ACB98CBAACB4DCB57CB30EA
S123C080CB60D730D6DCD706D71ED743D756D768D773D78BD7B0D7C0D761D7DBD7EFD7FA15
S123C0A0D7D0D805D810D81BD82DD83BD849D6EBD871D896D881D857DCB9DD97DD9BDDE0A6
S111C0C0DA44CB63CB6CDA1DDA53DA64000089
S123C5000101010101CC0000FDFF028EFEFF7F003C8D21B67F0084C088C027037EC6CAB6A5
S123C52080004A26F7CC8001CEC300ED008600A7097EC6CACE002A4FA700088C003926F828
S123C540CE1000860AB77F00970E86FF9722972397249725CC07C0DD261C39801D282086C9
S123C560B0A72B860CA72D86079739BDDB38CC0000DD0CDD12DD148608970BCCC110DD164D
S123C580DD18DD1A8620B7C6B0CEC300C6208640A7098FC300108F5A26F6CEC300DF08CC40
S123C5A0C200ED00CCFE00ED04C30001ED02830100ED06860AA7088620A709EF0CEF0EDC7A
S123C5C00CC30001DD0CED0ABDDA64CEC5F2A6002706BDDB0A0820F6CE10001C200118CE93
S123C5E03000180926FC1D20011D0008CC0000DD2639496E74657261637469766520432058
S123C60020205620322E3836322028414B46290A008D6B8D74816125F881732604863E2019
S123C62068368D513C18388D4C328172270D8177270F816327118162271B39A6008D4A2077
S123C64010188FE700200A188FA400A700EA00E700863E2034188F373C32331B331B9701B3
S123C6605D270C8D19A7009B019701085A26F496018D1620DC8D07368D0416328F39B610C2
S123C6802E842027F9B6102F39F6102EC48027F9B7102F39DE08A608970A1AEE00EE02186A
S123C6A0E600F7C6A91808FCC000FDC6AEBDFFFF20ED8620B7C6B0DC088FED021AEF00A631
S123C6C00981402604EE0CDF0839963C260CCE10001F2E2005BDC61120F0120B02ECDE085F
S123C6E0EE0EDF088CC3002607DC1EC30001DD1EA609810026D4BDC694810027CD81402780
S123C700C9812027048602200286048D0220BB9701940B910126013996019A0B970B7EC697
S123C72089EC02A300201CEC02A400E4012014EC02AA00EA01200CEC02A800E8012004ECB6
S123C74000E302ED020808398D26A601E6033DDD00A600E6033DDB00D700EC013DDB00D701
S123C760007D000727064F5F930020D7DC0020D37F00078D6308088D5F090939BDC770EC60
S123C780023CEE0002DF003820D7EC00A3022705CC000020AECC000120A9EC02A3002EF5B8
S123C7A020EEEC02A3002DED20E63CEC002B1C26043808083937368605B7C7BFEC02380041
S123C7C027030926FA380808ED00394F5FA30037368604B7C7BF20E46D002A094F5FA3001A
S123C7E0ED007300073963006301394F5FA300ED0039EC002705CC0001ED0039EC0027F60A
S123C8004F5FED0039EC02E306DD00E601E905A600A904ED04DC00ED06C6043A39EC06A3D2
S123C82002DD00E605E201A604A20020E6EC06A302E605E201A604A2002D1E2025EC02A323
S123C84006E601E205A600A2042D0E2015EC06A302260FEC04A3002609C6063ACC0001EDF6
S123C8600039C6063ACC0000ED00397F0007BDC9093CC6043ABDC909CE0000DF0038A60311
S123C880E6073DDD02A603E6063DD301DD01960089009700A602E6073DD301DD01960089AE
S123C8A0009700A603E6053DD300DD00A602E6063DD300DD00A601E6073DD300DD00EC036B
S123C8C03DDB00D700A602E6053DDB00D700A601E6063DDB00D700A600E6073DDB00D700DF
S123C8E0C6043ADC02ED02DC00ED007D000727028D0139CC0000A302DD00C600E2018600A9
S123C900A200ED00DC00ED02396D002A058DE47300073918EC00180818080909ED0039182C
S123C920EC020909ED0018EC00180818081808180820E718E600183A18A60009A70018099C
S123C9405A26F518E600183A393CCDEE00E600384F20C38FCDEE00EE028F0909ED008FCD6A
S123C960EE00EE008F20AF18E6003C3AEC00DD00EC02380909ED00DC00209D18E6003C3A0A
S123C980EC003820933CA601CDEE00A70020083CEC00CDEE00ED0018083818080808393C82
S123C9A0EC00DD00EC02CDEE00ED02DC00ED0038C6043A57183A39EC00DD00EC02D707187E
S123C9C0E6003C3AD607ED02DC00ED0038080820C9EC00D70118E6003C3AD601ED0020B95C
S123C9E0A6013CEE02273FA70038202AA601B7C9F83CEE0227301C00FF38201AA601B7CA7A
S123CA00083CEE0227201D00FF38200AEC003CEE022713ED00380808080839EC00DD00EC94
S123CA20023CEE0426063886057EDDECED02DC00ED0038080820DFEC003CEE0227E8E7007F
S123CA4038ED02080839EC003CEE0227D9ED0038ED02080839EC00DD00EC023CEE0427C61B
S123CA60ED02DC00ED0038EC02ED04DC00ED020808393CEE0027AFE6004F38ED00393CEE12
S123CA800027A3EC0038ED00393CEE002798EC00DD00EC02380909ED02DC00ED003918EE9D
S123CAA000391AEE00080839EC00260618EE0008083918081808080839EC0026EF20F3ECF8
S123CAC00027EFCC0001ED0018EE0039EC0026E218EE0039EC00DD0018EC00DF04D3048FFA
S123CAE01AEE002705DC00ED0039DE088640A7098621B7C6B0EC0C1AEE0E8FCDEF0C1AEF5E
S123CB000E3918EC00DF00D3008F1AEE0027DB080839EC00DD00EC02DD0218EC00DF04D3E2
S123CB20048F1AEE0227C3DC00ED00DC02ED0239DF00DE08DC00A306CDA30025071808187D
S123CB4008DE00391809DE0086047EDDEC8F18E3008F18081808393C323318E3007EC91657
S123CB60EE0039EC00DD3A0808180839DC3A0909ED00180839EC003CEE021AA30038242758
S123CB80E302C30002ED02080839EC003CEE021AA3003824120520E8EC003CEE021AA3008A
S123CBA0382404050520D97EDDE6EC003CEE021AA3003824F218A60018083D20C33CBDD6DD
S123CBC04DCE00003CDF3DDF3F7F00411830CDEE06A600BDCD152528812D260B73004108CA
S123CBE0A600BDCD152519812E260B08A600BDCD1524037ECC833131BDD65638860F0D392F
S123CC00A600BDCD152477BDCC940824F37C003DA60008BDCD1525F5812E260AA600BDCDC5
S123CC201524030820F681452707816527037ECCD708A600BDCD152515812D2706812B273C
S123CC400520B318630008A600BDCD1524A8803018A70108A600BDCD15241418E6015858C0
S123CC6018EB015880301B18A701088126228718A601186D002A01409B3D973D2059812EEE
S123CC8026A408A600BDCD15249C8D0808258D7A003D20EF963E9743DC3FDD440579003EFE
S123CCA0252C0579003E2526D34436963E9943973E32251A0579003EDD3F2512E600C030F0
S123CCC04FD33FDD3F963E89002503973E39DC44DD3F9643973E39CDEF06CE003DBDCD4086
S123CCE0272C963D18A7018696973DBDCD21186D01271B2A0BCECD4BBDD67F18600120061B
S123CD00CECD4FBDD67FBDCD5F186A0126F83131BDD656383981302506813922020D390CC1
S123CD2039CE003D8D1A27147D003E2B0FDC3F7A003D270A0579003E2AF5DD3F0C390D394F
S123CD403736EC002602EC023233393DCCCCCD41200000BDCFFBBDD64DBDCECABDD6567D9D
S123CD60003D27057D0042260ACC00009741DD3DDD3F39964198469741963D9B422A0924B0
S123CD80168606CEFFFF2009250D8607CE0000DF40DF3DDF3F0D398B82973DCE00003C3CA5
S123CDA030BDCDD86D002B0B69036902690169007A003D6D032A13A6024CA702260CC60196
S123CDC0E3002404467C003DED0038DF3E329740317D003D27B45F399645D6403DA7019630
S123CDE044D6403DE300ED009645D63F3DE300A70324026C026F006F019643D6403DE3028A
S123CE00ED029644D63F3DE302ED0224026C019645D63E3DE302ED0224026C019643D63F0B
S123CE203DE301ED0124026C009644D63E3DE301ED0124026C009643D63E3DE300ED00398B
S123CE40BDD64DCED37ABDD67F7D00412703730046BDCEFCBDD6564FD63DC17F24035F2068
S123CE601B53C3FF902F178FDC3E2001040926FC7D00412A074353C300012A020C39860966
S123CE800D39CC0000DD004FD63DC17F24035F203353C3FFA02F2F8F96405FDD00DC3E2036
S123CEA007047600007600010926F67D00412A147300007300014353DE0008DF002605C325
S123CEC000012A020C3986090D39BDD2E2CE0045964280972A1BC6038B082A096F00095AEE
S123CEE026F66F0039C6804A2B035720FAE400E7008D028D07964688FF974639963D260ECD
S123CF00DC42DD3DDC44DD3F964697415F397D004227F9D641D84690422510811822ED1872
S123CF203C36CE004318CE003E201740811822D0183C369642973D96469741CE003E18CE68
S123CF40004317363636A8003617A8013617A8023630A606E7061684074CC4185454543A3E
S123CF60E6034A27095666026601660020F45618A602A900974018A601A901973F18A60018
S123CF80A902973E30A6062B15245A76003E76003F7600407C003D264CCCCD812053251B5C
S123CFA073004170004024087C003F26037C003E70003F24037C003E70003E7D003E2B25F6
S123CFC02613963D80082326973DDC3F27207F0040DD3E20E67A003D271478004079003FF8
S123CFE079003E2AF01AEE07C6093A355F39CCCD8A1AEE07ED07C6073A3539964698419790
S123D000417D0042260586087ECD837D003D26055F7F004139963D904224052B057ECD8A75
S123D0202B1F8B7E973DDC3E93432B182606964090452B10DC3E04760040DD3E7C003D26B2
S123D040037ECD81DC3EDE430826010903183C18DE3EDF3E3CCE00003C3C309645D63F3D03
S123D060A703BDCE0218DF3EDC3FA301DE4303DF3F7F003E383832331838D33EDD3E5F3999
S123D0803CCE003DBDCD40260738CC3000ED0039DE3D3CDE3F3C964136BDD64DCE00003C4D
S123D0A03C3C1830CDEE0F86207D004127057F0041862DA70008CDEF00CED1EABDD67FBD1C
S123D0C0D1EE2E19CED1E6BDD67FBDD1EE2E16186A02CECD4FBDD67FBDCD5F20DC186C0204
S123D0E0CECD4B20F0CED37ABDD67FBDCEFCD63DC07F50CB17200A74003E76003F760040B7
S123D1005A26F4860118A70318A6028B082B0A810824064A18A7038602800218A702186DB7
S123D120032E15862ECDEE00A70008186D0327058630A70008CDEF00CED1D1860718A705F1
S123D140186F04DC3FA301DD3F963EA200973E2505186C0420EDDC3FE301DD3F963EA900C3
S123D160973E18A6048B303CCDEE00A70008186A032605862EA70008CDEF0038080808187C
S123D1806A0526BCCDEE0009A600813027F90818E602272A8645A70008862BA7005D2A0548
S123D1A050862DA70008CDEF004FCE000A02378FCB30CDEE00E7000833CB30E700086F00DD
S123D1C0383838BDD65632974138DF3F38DF3D38390F42400186A00027100003E800006457
S123D1E000000A000001497423FE4B18967F96462A12D6412A0EDC421A933D2617DC441AE4
S123D200933F20109141260CDC3D1A93422605DC3F1A93440784F424028A080639CE008EF3
S123D220C3000026057ECD8A09052AFCDD3E7F00408F9741D73D5F394D2AE24353C3000153
S123D240CEFF8E20DBCE009EC30000261118DE0026037ECD8A0978000179000059492AF55E
S123D260DD3E960097408F9741D73D5F394D2AD57300007300014353DE0008DF002603C395
S123D2800001CEFF9E20C1CE003DBDCD402601397D00412A04860A0D39BDD64D860436DEC8
S123D2A03F3CDE3D3C18308D399642807E4C2A03442003448B7E9742BDCFFBBDCEFC7A0026
S123D2C03D8D1F18EC00DD3D18EC02DD3F186A0426E6DC42DD3DDC44DD3F383831BDD65691
S123D2E05F39DC3DDD42DC3FDD449641974639BDD64DCED449BDD67FBDCFFBBDD656DC3DCB
S123D3001A8385B32B0B7D004126037ECD817ECD8ABDD64D9641367F0041BDCECADC42272F
S123D320068086544C26FC5C37CED35EBDD60DCED35ABDD67F2003BDCD5F306A0026F832E6
S123D340324D2A0CBDD2E2CED5A2BDD666BDCFFBBDD6565F39BDD64D20EA402DF85436384C
S123D360EF1D37D00D0139500D013AB60B613C0888893D2AAAAB3E2AAAAB3F0000003F80C9
S123D38000003F800000FFBDD3A3BDCD5F7ED2FE8D11BDD64DCED449BDD67FBDCD5FBDD66A
S123D3A0565F3996412704860C0D39963D27F8BDD64D3C3C30BDD6974FD63DC07F2A0143EE
S123D3C0BDD238CED445BDD67FBDCD5F30BDD67FBDD697867F97423C3C30BDD6A5CED5A231
S123D3E0BDD666BDCEFC30BDD67FBDD697CED441BDD666BDCEFC30BDD67FBDCFFB30BDD64E
S123D40097BDD2E2BDCD5FCED424BDD60D30BDD67FBDCD5F383830BDD67FBDCEFC3838BD20
S123D420D6565F393E1D89D93E3A2E8C3E638E393E9249253ECCCCCD3F2AAAAB40000000EE
S123D440FFBF8000003F3172183EDE5BD9860E0D39860D0D39BDD64D9641367F0041CED53D
S123D460A2BDD67FBDD1EE2F07BDD35586FF20014F363C3C30BDD697BDD2E2BDCD5FCED464
S123D480ACBDD60D30BDD67FBDCD5F3838324D270CCED4A8BDD67F730041BDCEFCBDD5F8CE
S123D4A0329741BDD6565F393FC90FDBBCE2DD1B3D70F0F1BD8888893D9D89D9BDBA2E8C04
S123D4C03DE38E39BE1249253E4CCCCDBEAAAAAB3F800000FFBDD64D4F2005BDD64D86F0DB
S123D4E036CED5C0BDD67F2003BDCEFC964126F92003BDCEF1BDD1EE2EF88D61240930A6AB
S123D500002B04880FA7008D54240930A6002A04880FA7008D47240730A60088F0A700CE88
S123D520D605BDD67FBDCD5FBDD2E2BDCD5F3C3C30BDD6A5A6042A05CED5A72003CED5925C
S123D540BDD60D30A6044724037300414D2B06BDD67FBDCD5F383831BDD6565F397A0042D4
S123D560BDD1EE2E020C397C0042730041BDCEFC7A00420D39BDCECADC3DDE42DD42DF3DF2
S123D580DC3FDE44DD44DF3F9641D6469746D7415F393638EF1DB9500D013C088889BE2ABD
S123D5A0AAAB3F800000FF37D00D01BAB60B613D2AAAABBF0000003F800000FF40490FDBB7
S123D5C043B40000BDD64DBDD2E2BDD4DBBDD578BDD4D5BDCFFB2407BDD656860B0D39BDF4
S123D5E0D6565F397FFFFFFFBDD64DCED605BDD67FBDCD5FBDD65639BDD64DCED60920EEA6
S123D600CED5BC20613C8EFA3142652EE18FDE3D3CDE3F3C8F9641363CCC0000DD3DDD3F62
S123D620DD40201030A6029746EC03DD44EC05DD42BDCD5F30EE00BDD67FBDCEFC38C60422
S123D6403A3CA6004326DD30C6073A3539383C3C8F303736204F300808BDD67F3831313157
S123D660316E00CED5A27F0041EC02DD3FEC00052403730041973D27020D56D73E5F397FA0
S123D6800046EC02DD44EC00052403730046974227020D56D74339DC3FED02DC3D58D1411B
S123D6A04656ED0039DC44ED02DC4258D1464656ED00397F00415F397D003E2705CC7F803C
S123D6C0DD3D4F5FDD3F397D003E27037300415F39BDD67F08080808BDD666393C183CEC18
S123D6E000BDD238183838090920AC3C183C0808BDD6660909EE00BDD080183838EC00EDF2
S123D7000408080808393C183CBDD666BDCE8218383824037EDDECED00DC00ED02393C18D7
S123D7203CEC02DD00EC00BDD26D1838387ED6973C183CBDD666BDCE5718383824037EDD0E
S123D740EC205D3C183CBDD6D1BDCEFC183838080808087ED6973C183CBDD6D1BDCEF120BE
S123D760EBA6008880A700393C183CBDD6D1BDCD5F20093C183CBDD6D1BDCFFB18383824FF
S123D780037EDDEC080808087ED6973C183CBDD6D1BDD1EE183838260CCC00010808080819
S123D7A00808ED00390808080808086F006F01393C183CBDD6D1BDD1EE1838382BDB20E5E4
S123D7C03C183CBDD6D1BDD1EE1838382ECB20D53C183CBDD6D1BDD38720A13C183CBDD670
S123D7E066BDD28718383824037EDDEC7ED6973C183CBDD666BDD2FE20EA3C183CBDD6661F
S123D800BDD2EF20DF3C183CBDD666BDD3A320D43C183CBDD666BDD39020C93C183CBDD622
S123D82066BDD4550736BDD5E8320620B73C183CBDD666BDD5F8BDD4D520A93C183CBDD66D
S123D84066BDD5F8BDD4DB209B3C183CBDD666BDD5F8BDD5C4208D8602E6019D4A080839F8
S123D860BDDB57A600BDDC45A601BDDC4508082003BDDB57A600BDDC45A601BDDC45080871
S123D88039BDDB573CEE008602E60027059D4A0820F738080839183CDF00BDDAB01A8300FA
S123D8A051240C8621B7C6B0DE001838180939DE00DC00C30002E300DD02830002DD04DE02
S123D8C002EE000808A60026037EDA0B812527037ED9F908A6008166261BDF02DE04090947
S123D8E03CBDD666380909DF04CEC100BDD080CEC1007ED9EB8164267DDF0218CEC100DE67
S123D900040909DF04EC022A0C862D18A7001808CC0000A302CE000A02378FCE000A023732
S123D9208FCE000A02378FCE000A02378FCE000A0237183C388601335D27064FCB30E70002
S123D94008334D27045D27064FCB30E70008334D27045D27064FCB30E70008334D27045DD7
S123D96027064FCB30E7000833CB30E700085FE700CEC10020758178262ADF02DE04090998
S123D980DF04A602BDDC2BBDDAF8257217BDDAF8256CA603BDDC2BBDDAF8256217BDDAF8AE
S123D9A0255C206181632611DF02DE040909DF04A603BDDAF82547204C8162261EDF02DE98
S123D9C0040909DF04E60318CE00085886308900BDDAF82529180926F2202A8173261ADF69
S123D9E002DE040909DF04EE020808A6002708BDDAF8250A0820F4200CBDDAF82409860A23
S123DA00BDDB0A2006DE02087ED8C5DE00DC00C30002E3008FCC0000ED001838393CDC14D8
S123DA20C300011A931426FBC30001CE0000081A931426FA8F380909ED00CC000C0909ED24
S123DA40007EC748090909090FDC14ED02DC120EED0039EC0008083C183CEE00AD0018388A
S123DA6038ED00390F3C183CB6103C84402605CEFF002003CEBF003CC6C03A18CEE0C41A97
S123DA80EF0008083C32324D26F538CCC500EDFECCDE64EDE2CCDE57EDE0CE10006F226F3E
S123DAA0248630A7211C23181C22181838380E39960B84082707CC00F0DD062016DC18938D
S123DAC0162307830001DD062009CC00F09316D318DD06960B84102705CC00F02012DC1AFA
S123DAE0931623058300012007CC00F09316D31A1A93062302DC06393736BDDAB01A830010
S123DB000224040D323339322001370F3CDE16088CC2002603CEC110DF16A700960B84087C
S123DB2027119C18260DDE18088CC2002603CEC110DF1838330C0E39BDDBD1CC00389D4AA5
S123DB408D2FC60C9D4A8D298D308D258601970F8608971C4F971DCC00019D4A8D13C60696
S123DB609D4A8D0DC68F9D4A8D073918CE011E200418CE0B29180926FC39CC00409D4A86DF
S123DB8002CEDB91E6009D4A8DE1088CDBD126F43900060F1C181C0F0600001111110F01BA
S123DBA00E00000000000C040800000F11110F010E00000C0C000C0C0000000C0C000C0494
S123DBC008020006020202120C00000E1F1F1F0E00CEDBE618CE004AA60018A70008180848
S123DBE08CDC2B26F339DF47CE10000F1D3C201D001097496F078104260E8601A7041C0026
S123DC0010A6031D0010201C8601A7041C0010A6031D001086FFA7079649A704E7031C00E7
S123DC20101D00101C3C20DE470E3936840F8B30813A2B028B071632444444448B30813AF3
S123DC402B028B0739BDDC2B371686029D4A339D4A39CE000A02378FCE000A02378FCE00E7
S123DC600A02378FCE000A02378FCE000A02379D4ACC00019D4ACC00079D4ACC008F9D4A86
S123DC80860233CB309D4A33CB309D4AC62E9D4A33CB309D4A33CB309D4A33CB309D4AC6EE
S123DCA06D9D4AC6739D4A39CC00029D4A8602E60027059D4A0820F739183CDF00CC7FFFA8
S123DCC0DD04CEC3001AEE0E188CC3002607CCE400DD06200518EC04DD06EC0693063CDEDC
S123DCE000A300382B091A93042E04DF02DD04188CC3002705183C3820CBDC041A837FFF67
S123DD00260486012015CEC310A609814027158FC300108F8C620026F08602DE0018381809
S123DD20097EDDEC3C1838DE02EE0E1AEF0CCDEF0EDE021AEF0ECDEF0CEC0683000118ED0E
S123DD4004C30001DE00A30018ED06A60318A708EC0418ED00860018A709DC0CC30001DD2F
S123DD600C18ED0ADC00E306C30008EE068F09DF0018DF0218EE0436A60018A70032091898
S123DD800983000126F1DE0218081AEF02DE0009DC0CED00183839862020513CEC00DD006F
S123DDA0CEC300EC0A1A9300270EEE0E8CC30026F238CC0001ED00399C082604387ECAEA30
S123DDC0183C8640A7098621B7C6B0EC0C1AEE0E8FCDEF0C1AEF0E183838CC0000ED0039AB
S123DDE08621B7C6B0391809860320003CDE084D2602861FA70997018621B7C6B0960181D8
S123DE00202431CEDE36A6002708BDDAF825F70820F44FD601C00A25034C20F9CB0A8B30FE
S123DE20BDDAF825FB178B30BDDAF825FB860ABDDAF825FB38390A52554E54494D4520456B
S123DE4052522000CE1000DC28E316ED161D237FA6008880A7003BCE1000DC26E31EED1EE1
S123DE601D23F73BCE1000CC07D0E31CED1C1D23EFA62236A7220EDE1408DF142605DE1297
S123DE8008DF127A000A26058621B7C6B086049D4A848027037EDF6F9615843F2640960F1E
S123DEA08101223A0F4FC6CF9D4ADC1E1A8300642D0BCC0000DD1E961C880C971C961C847D
S123DEC0082704C6002002C60786029D4A4FD611C1102502CB30CA809D4A0E7EDF6F9639E4
S123DEE0840126037EDF6F960F8102245EDE1A9C16277C088CC2002603CEC110DF1AE600B0
S123DF00960F81002634C10A26068601970F205F9611811F27594C9711811126074F37C614
S123DF20C09D4A33C120250CC17F2208CEDFD1C0203AE60086029D4A20358101260DD710A9
S123DF40FCDFBF9D4A8602970F2024810A2712CEDFBFD60F3AEC009D4A960F8B02970F20B0
S123DF600E8600970F86019711D610C10A26B5D60E96398404273E96224824068B01C8107A
S123DF802002CA10972296234824068B01C8202002CA20972396244824068B01C840200281
S123DFA0CA40972496254824068B01C8802002CA809725C8F0F77F0032CE1000A7223B002D
S123DFC001000600CF020000020011495557777FFF202122232425262728292A2B022D2E49
S123DFE02F3031323334353637383904053C3D3E3F404142434445464748494A4B4C4D4EB9
S123E0004F505152535455565758595A5B5C5D5E5F60616263646566036869066B6C6D6EF4
S123E0206FF0F172737475767778017A7B7C7D7E7F18CE03E8180926FCCE10001F00043325
S123E040CC1BE61F00042C83000126F7203937368D56CC00029D4ACEE07C8602E6002705DD
S123E0609D4A0820F732BDDC4532BDDC458602C6299D4ACE10001C28204F06CF2A48616C73
S123E0807465642A2028008D1FCEE098BDDCA8CE10001D23FB8D163B2D504F574552204782
S123E0A04C495443482D20008601978D39860E978D39CE80004F5FE3008FC300028F8CFF79
S108E0C00226F4393BC7
S123BFC0E0C4E0C4E0C4E0C4E0C4E0C4E0C4E0C4E0C4E0C4E0C4E0C4E0C4E0C4E0C4E0C41D
S123BFE0DE57DE64E0C4E0C4E0C4E0C4E0C4E031E0C4E0C4E0C4E0C4E0C4E0C4E0C4C50040
S123FFC0E0C4E0C4E0C4E0C4E0C4E0C4E0C4E0C4E0C4E0C4E0C4E0C4E0C4E0C4E0C4E0C4DD
S123FFE0DE57DE64E0C4E0C4E0C4E0C4E0C4E031E0C4E0C4E0C4E0C4E0C4E0C4E0C4C50000
S105FF020000F9
S105FF000256A3
S9030000FC
